:0600000025006400000B66
:04000C0008022200C4
:10001000A7070D0C280000000008A706120C2800F6
:100020002F040008A706E904170C28000008090798
:100030002F051C0C280000082903E905210C2800C5
:100040000008120C2F06260C28000008A706E90459
:100050002B0C280000082D0C290A09022A00320C5A
:1000600028000008FF0C2900370C28000008A7070B
:100070000F05080C28000008000C8A01450C0F062B
:1000800043073C0C2B000F04230B000C8A014E0C81
:100090000F064306450C2B000F04230B800C8A012E
:1000A000980E570C43073C0C2B000000230B690CE7
:1000B000CA06600C2B000A02070E100D2400230B49
:1000C0000F063C0C2B000A020F06EA070002200074
:1000D000230B3C0C2B0000027F0E64052000AA07B6
:0400E0006000230B8E
:10020000C70C020066006700380C0600200C0700CF
:10021000080C28003C0C2B00010C2D00400C300079
:1002200031003200330034003500360037007800EA
:1002300079007A007B007C007D007E007F006F00EB
:100240006C00FF0C29000609ED004306CD050D02E8
:100250009E006C030D029F006C030D029D006C0359
:100260000D029C006C0306090D029B004C03270045
:100270000D029A006C030D0299006C030D029800A8
:100280004C03070E26000609000000000B022200A6
:0207FE00380CB5
:021FFE00D10F01
:00000001FF
